:1000000064C0FECFFDCFFCCFFBCFFACFF9CFF8CF46
:10001000F7CF11C5F5CFF4CFF3CFF2CFF1CFF0CFBB
:10002000EFCFEECFEDCF000041A042A1E045A3A469
:10003000A5A64BA74D484FA8504354A9AA58E1ABD9
:10004000ACE2ADAE62AFB0B161B2B3B4E365B6B726
:10005000B8B9BABBBCBD6FBE7063BF79E478E5C008
:10006000C1E6C2C3C4C5C6C7556B7261696E65205F
:1000700032303134002A536F69722A002020206EFA
:1000800069676874206D6F646520003A00636F7261
:100090002E2074696D6500207365630020207475DF
:1000A0006E696E6720736F756E6420003030004893
:1000B0007A002020202045787465726E616C2020C3
:1000C00020000200020026000000F894EE27ECBB9E
:1000D000F1E0FBBFEBBFE5BFF8E1F1BDE1BD8DE0B5
:1000E000A2E0BB27ED938A95E9F780E094E0A0E6D3
:1000F000ED930197E9F7E2ECF0E085919591009797
:1001000061F0A591B59105901590BF01F0010590A2
:100110000D920197E1F7FB01F0CFEFE5EDBFE4E0D1
:10012000EEBFC0E6D1E0A7C4BA93AA931A93EB81BD
:10013000EE0FEE0FEE0FE064AE2F59D010E0183046
:1001400048F4A981BA81EE27A10FBE1FAC914AD015
:100150001F5FF5CFA0E84BD018812496089528970B
:1001600099D5E0E0EE83EF839ED5A0D5A2D5E0E05F
:10017000A6D5ABD59BD58ED5EFE1EE83EF83A8D581
:1001800095D5EFE1E883E983EA83EB8398D5A3D59E
:100190008DD58FD5ECE1EC83ED83EE83E0E0EF834A
:1001A0009DD584D528960895AA939BD5E07FA4D5A4
:1001B00098D5E295E07FA0D58BC2A4E1A7D5A5E0B4
:1001C000A5D58CED90E00197F1F7A3E0A3D5A2E0CF
:1001D000A6D5ACE29FD5ACE09DD5A1E0A0D5A6E028
:1001E00099D50895AA93909AA881DEDF71C2AA9347
:1001F0009098A881D9DF6CC2AA931A93EA8193D50B
:10020000309721F092D511F410EC01C010E8E9818B
:100210001E0FA12FECDF1881A8C11A9310E0103136
:1002200070F4E12F80D5E05AFE4FA0E2A083E12FC9
:100230007AD5E059FE4FA0E2A0831F5FF0CF6AC0DD
:10024000AA93E881E03041F4E52D6DD5E05AFE4FE8
:10025000A981A083539407C0E42D65D5E059FE4FD2
:10026000A981A0834394DDC2AA93EF97219780E4EC
:10027000A0E0B0E0E8E2F0E014D65BD5E491E03035
:1002800009F157D5A491A03C50F053D5E4914BD53A
:10029000E05CF040DE01AE0FBF1FEC9102C049D51B
:1002A000E491EA93DE01AF5BBF4FAC91C9DFDE01A1
:1002B000AF5BBF4FED91FD913196FE93EE93319779
:1002C000E491DBCFEF9624960895BA93AA931A93FC
:1002D000EC81EA93AC8190DF10E0103148F41F5FAD
:1002E000A981BA81ED91A983BA83AE2F7BDFF5CFC7
:1002F0001881259608951A9310E0E89420F8E6B73F
:10030000E07841F4143610F41F5F03C0689420F8BD
:1003100001C0F5CF19910895E4EEE6BFECDF089532
:10032000AA93E881E3B9E4E8E6BFE5DFD1C1AA9387
:100330001A93A981A13011F4E4EC01C0E4E8E6BF0E
:10034000DADF13B1E12F18816CC2E4E9E6BF08954A
:10035000AA93EA81E370EA83E981E03019F0EA8147
:10036000E061EA83E881E03019F0EA81E068EA833D
:10037000E7D4A7E0D5DFAA81D3DFE7DFF6C0AA93F1
:10038000DFD4A0E0CDDFA881DED4A981DCD4AA81AE
:10039000DAD4DBDFEAC0D4D4A0E0D8D4DBD49E2EFC
:1003A000D9D46E2ED7D47E2EA0E0C1DFAE2F5BD481
:1003B0008E2ECBDF0895AA931A93C2D4A981C6D4F6
:1003C000A0E0B5DF1E2FC1DFE12F18812AC2AA935A
:1003D000B7D4A981A5DFA881A3DFB7DF22C2E1E3FB
:1003E000BE1610F4B39415C0BB24689421F8E9E05C
:1003F000AE1610F4A39403C0AA24689422F8E5E092
:10040000EA1511F4689423F8E9E0EA1511F4E89488
:1004100023F80895772091F4662071F4EEE1E91550
:1004200051F424FE08C0E0918101E90DE9519E2EAE
:10043000E89424F893D402C0689424F80895AA9309
:10044000E88171D4309711F4E0E342C16ED411F425
:10045000E1E33EC1E230A0E0FA0711F4E2E338C183
:10046000E330A0E0FA0711F4E3E332C1E430A0E0A6
:10047000FA0711F4E4E32CC1E530A0E0FA0711F427
:10048000E5E326C1E630A0E0FA0711F4E6E320C177
:10049000E730A0E0FA0711F4E7E31AC1E830A0E082
:1004A000FA0711F4E8E314C1E930A0E0FA0711F407
:1004B000E9E30EC1E031A0E0FA0711F4E0E208C17F
:1004C00007C1A0E1B0E0E0E0C9D4A1E0B0E0E09174
:1004D0008B01C4D4A2E0B0E0E0918A01BFD4A3E0D4
:1004E000B0E0E0918D01BAD4A4E0B0E0E0918C01DD
:1004F000B5D4A5E0B0E0E0918101B0D4A6E0B0E0D1
:10050000E0918501ABD4A7E0B0E0E0918401A6D4EE
:100510000895AA93999913C0E881AA81AE1718F497
:10052000EA81EF5F01C0E981EA831CD4A13011F0B8
:100530001CD419F4689431F802C0689432F89A997E
:1005400013C0E981AA81EA1718F4EA81E15001C0D9
:10055000E881EA8307D4A13011F007D419F4689434
:1005600031F802C0689432F8EA8123960895989988
:1005700002C030FE01C00CC0689430F8F3D3A9303B
:1005800020F4E0918801EF5F01C0E0E0E093880192
:10059000E9D3A13029F46A92EBD3ABE3BADF6E2E34
:1005A000E4D329F47A92E4D3A7E1B3DF7E2EDAD341
:1005B000A33031F4999B02C09A9902C09924CED3FA
:1005C00031FE03C0CBD3E89431F8CCD3A43039F456
:1005D000E0918A01D0D3ABE39CDFE0938A01C2D3E0
:1005E000A53039F4E0918B01C6D3A7E192DFE09307
:1005F0008B01B8D3A63039F4E0918C01BCD3ABE3C6
:1006000088DFE0938C01AED3A73039F4E0918D01FF
:10061000B2D3A7E17EDFE0938D01A4D3A83039F4F3
:10062000E0918101A8D3A2E374DFE09381019AD322
:10063000A93069F4E09184019ED3A4E66ADF73D304
:10064000E0938401F093850198D308F49CD3089536
:10065000989B04C0999B02C09A9926C09ED3E0E063
:10066000E0938901A0918601AF3F28F4E0918601D3
:10067000EF5FE0938601A0918601A43121F477DF3A
:10068000E1E0E0938301A0918601AB3F60F0A0918F
:100690008701A43620F4E0918701EF5F02C067DF95
:1006A000E0E0E093870107C0E0E0E0938701E0939A
:1006B0008601E89430F80895AA93CC24DD24A8811B
:1006C000AA3028F0E881EA50E883C394F8CFD880B4
:1006D0002196089555244CD35A92A0E6B1E0F5DD59
:1006E0004424E1D24A92A0E7B1E0EFDD0895E2E0D0
:1006F0005E2EE8E6F0E056D358D3E5E04E2EE5E76F
:10070000F0E055D30895AA93A881A33019F4A091DD
:10071000800150D3AC2D4ED3AD2D4CD382C0AA93C3
:1007200058804880E981FFD2309741F4D4D246D333
:10073000BAD244D3D0D242D3E4E06BC0F6D251F463
:10074000B2D23CD3C8D23AD3C0D23AD3C4D238D32F
:10075000E2E065C0E230A0E0FA0761F4B9D22ED33E
:10076000B7D22CD3B8D22AD3B6D22AD3AED228D37A
:10077000E2E055C0E330A0E0FA0711F4E3E041C045
:10078000E430A0E0FA0751F4A6D218D39ED216D3D3
:10079000A2D214D3E0E216D3E0E23EC0E530A0E0FE
:1007A000FA0731F498D20AD393D208D3E3E02EC0EB
:1007B000E630A0E0FA0741F48ED200D389D2FED20F
:1007C00087D2FCD2E4E025C0E730A0E0FA0741F48C
:1007D0006AD2F4D268D2F2D27ED2F0D2E0E21CC069
:1007E000E830A0E0FA0741F476D2E8D271D2E6D23E
:1007F00072D2E4D2E4E00DC0E930A0E0FA0789F457
:10080000E4E0EA93DBD264D2D9D2E4E0EA93D6D230
:10081000E2E0EA93D5D2E2E0EA93D2D2E4E0EA93CE
:10082000CFD22296089533FE06C0E0E1DE2ECCD270
:10083000E0E1E09380010895F0DC5524442423FE98
:1008400004C0999B02C09A9901C002C0689401C07B
:10085000E89433F887D2A330A8F4A72DB8D209F4CE
:10086000B3D283D209F4DFDFB5D223FE04C0B8D2FD
:10087000A5D234D2A5D2A62D1FDF74D2A13009F49F
:10088000D2DFB2D26FD2A33059F4A62D15DFA2D297
:10089000A7D294D223D294D2A92D0EDFC4DFA4D242
:1008A00061D2A43018F05ED2A83008F038C0ECE76E
:1008B000F0E078D27AD2A0918B0189D209F484D267
:1008C00051D2A53009F4AFDFE9ED7CD2ECD192D260
:1008D000A0918A01F1DE46D2A43009F4A4DFEBE84E
:1008E000F0E065D2E0D186D2EAE04E2EEAED6AD29F
:1008F000A0918D016CD209F467D234D2A73009F4EB
:1009000092DFD1D177D2A0918C01D6DE2BD2A63046
:1009100009F489DFEBE8F0E04AD2C5D16BD222D2EC
:10092000A83009F5E3E05E2EEDE8F0E03BD23DD2E1
:10093000E4E04E2EA0918101A93120F0A951BCDE46
:10094000439408C0A0918101E9E1EA1BAE2FB4DE17
:10095000EDE238D2CC2009F437D265DFA4D14AD2F7
:10096000E7E9F0E024D2FED1A93091F5ECE9F0E01E
:1009700019D21BD202D220F5A0918401B091850139
:10098000A436E0E0BE0748F4A091840120D209F427
:100990001BD2E0E1E093800105C0E1E0E09380013B
:1009A000CC24DD2440DF7FD1A3E0ADDE33FC03C0E7
:1009B000ECEAF0E0FCD1E6E04E2EEFEAF0E004C015
:1009C00033FC06C0E2EBF0E0FA93EA93A1E04CDCE2
:1009D0000895219758D2E0E0EE83A0918B010CD2CC
:1009E000E0918A010ED29F01A0918D0105D2E09184
:1009F0008C0107D2AF01A72DFFD1E62D02D28F01C6
:100A0000A0918201A13010F0E1E0EE8302171307FC
:100A100018F40417150720F4E1E0EE83689401C090
:100A2000E89427F8AE81A13010F0929A01C0929814
:100A300031D2279608950A921A92FA926A937A937B
:100A40008A939A93AA93BA93EA93FA93EFB7EA93A5
:100A5000E6E0E2BFC4DC689434F8E991EFBFF991B5
:100A6000E991B991A9919991899179916991F990B7
:100A7000199009901895E0E0E2BBEFEFE1BBE3E0ED
:100A8000E7BBE0E0E8BBE4BBEFEFE5BBE6E0E2BFDD
:100A9000E3E0E3BFE0E0EFBDE2E1EEBDE0E0EDBDAD
:100AA000ECBDE7BDE6BDE0E0F0E0FBBDEABDE9BDC1
:100AB000E8BDE2BDE5BDE4BDE3BDE1E0E9BFE0E0E6
:100AC000EAB9E0E8E8B9E0E0E0BFE0ECE7B9379A7E
:100AD000329A319AE0E0EDB9ECE0E0B9E0E0E2B959
:100AE000E4E0E6BFE0E0E1B943D142D1A0E030DC90
:100AF000A0E061DC1E2F1F773BD1A12F68DCA2E1B3
:100B00005ADCE13020F0E2E1EA93A0E060DCA0E111
:100B1000B0E098D1E03031F5A1E0B0E093D1E093BE
:100B20008B01A2E0B0E08ED1E0938A01A3E0B0E0B7
:100B300089D1E0938D01A4E0B0E084D1E0938C01F1
:100B4000A5E0B0E07FD1E0938101A6E0B0E07AD1EA
:100B5000FE2FE0E00F01A7E0B0E074D1E4D0E00D9B
:100B6000F11D11C0E5E1E0938B01E0E0E0938A0123
:100B7000E6E0E0938D01E0E0E0938C01E9E1E093B1
:100B80008101EAE0F0E0E0938401F093850105D172
:100B9000FAD0689424F8789410DBE1DA3EDBA7DD24
:100BA00099DDACE6B7E031D134FE03C0E89434F807
:100BB0004FDD21FE36C0E89421F8EDDB2BDC3CDE76
:100BC00089DD662059F425FC02C027FE01C005C05E
:100BD000689425F8E3E0E093830102C0E89425F8E7
:100BE000A0918301A130C0F0E0918301E150E09336
:100BF0008301E0E42E2626FE0BC0E0918401F091F3
:100C00008501309711F4C19A02C0E3E4EFBD03C03F
:100C1000E0E0EFBDC19805C0E0E0EFBDE89426F844
:100C2000C19822FE1EC0E89422F8D3DEA091820172
:100C3000A13028F0E0918201E150E0938201A0917F
:100C40008901AA3030F4E0918901EF5FE0938901D6
:100C500008C032FE03C035DCE89432F8E0E0E093EF
:100C60008801A2CFFFCFAA93E881E295EF70AE2F63
:100C7000AA0FAA0FEA0FEE0FA991AF70EA0F08951D
:100C8000AA93A991EE27AA5012F0E05FFCCFA65FCD
:100C9000EA0F0895EFE1E883E983EA83E0E0EB837C
:100CA000EC83ED830895E1E0EA930895DE01119667
:100CB0003BCAE0E0E883E983EA83EB830895EC83B1
:100CC000EFE1ED83EE83EF830895E2E0EA93089588
:100CD000E3E0EA930895E4E0EA930895E5E0EA9317
:100CE0000895919A88E28A95F1F7E2B3EF70E2BB3A
:100CF000E2B3AE2FE8810895EA2BE2BB88E28A9541
:100D0000F1F7919888E28A95F1F70895B0E07DD0E7
:100D1000A3E06DCA6CDA85E88A95F1F7089567DA81
:100D2000A2E0B0E072C0F0E00895E130A0E0FA0780
:100D30000895FE01EF5BFF4F0190F081E02D0895D3
:100D4000EBDAA0EDEDCA9CDFAE2FEACAE9DAE4DA0D
:100D5000A1EDE6CAA1E0EBDAAE2F85CF7A926A92D6
:100D6000A92D0DCBA09188010895FCDFA230089534
:100D7000E0E0EA930895EA93FBCFA0918401B0915B
:100D800085017DD00895E0918401F0918501A4EC66
:100D9000B9E045D0FBBDEABD0895EDE1E0938201E5
:100DA000929A0895FA93EA930895A0E05DCAFADF53
:100DB000A1E05ACA44DBEA93AA8142CAA0E040CA31
:100DC000A1E03ECAEA93FCCFE0E1CE2E089574DCA8
:100DD000CC200895CA92A0E0A2DCDA92A4E09FCCD5
:100DE000E8E05E2E4E2E7ACFCA92A9E098DCDA9225
:100DF000ADE095CCA2E087CCECE3EA9FF001DF0107
:100E0000089591DFEA0FFB1F0895109639F080EDE9
:100E100097E00197F1F7A8951197C9F70895002475
:100E2000112490E1AA0FBB1F001C111C0E1A1F0AEF
:100E300018F40E0E1F1E01C0A1609A9599F7FD01CE
:100E4000D0010895E199FECFFF93FFB7F894AEBBB0
:100E5000BFBBE09AEDB3FFBFFF910895E19B02C0D5
:100E6000A895FCCF9FB7F894AEBBBFBBE09A8DB3FB
:100E7000E81719F0EDBBE29AE19A9FBF08950024AC
:100E80000A160B0608955A934A933A932A931A9393
:100E90000A9308955D814C813B812A8119810881E3
:100EA0000895AC0FBD1F05900D928A95E1F7089546
:00000001FF
